:100000000C9451030C9489030C9489030C940E2CCA
:100010000C9489030C9489030C9489030C94890330
:100020000C9489030C9489030C944B2A0C94232B75
:100030000C94002A0C9489030C9489030C94890372
:100040000C9489030C9489030C9489030C94890300
:100050000C9489030C94272A0C9489030C9489032B
:100060000C9489030C9489030C9489030C948903E0
:100070000C9489030C9489030C9489030C948903D0
:100080000C9489030C9489030C9489030C948903C0
:100090000C9489030C9489030C9489030C948903B0
:1000A0000C9489030C9489030C94890305010902BB
:1000B000A10185020901A1000509190129081500FE
:1000C0002501950875018102050109300931158165
:1000D000257F95027508810609381581257F9501D0
:1000E00075088106050C0A38021581257F95017572
:1000F000088106C0C005010980A101850319012AF4
:10010000B700150126B700950175108100C0050CD8
:100110000901A101850419012AA002150126A002E6
:10012000950175108100C005010906A10105071997
:10013000E029E715002501950875018102950175F3
:100140000881010507190029FF150026FF00950603
:1001500075088100050819012905950575019102A9
:10016000950175039101C009023B00020100A0FA4C
:10017000090400000103010100092111010001220D
:100180004000070581030800010904010001030084
:100190000000092111010001227B000705820320D4
:1001A000000112010002000000081D8D3A34000118
:1001B0000102000124034100750072006F0072000B
:1001C0006100200043006F0072006E006500200097
:1001D00072006500760031000000180373007000A3
:1001E0006C00690074006B0062002E0063006F00F9
:1001F0006D0000000403090400000000000000007E
:1002000000000000000000000000000000000000EE
:100210000000000000000000000000007E0F00D47D
:10022000FFFFFFC700000078000000000000000092
:100230002A2B280000000000000000000000000041
:1002400000000029000000002C1E3420212224344C
:100250002627252E362D3738271E1F20212223241E
:1002600025263333362E37381F0405060708090ABA
:100270000B0C0D0E0F101112131415161718191A56
:100280001B1C1D2F3130232D350405060708090AD4
:100290000B0C0D0E0F101112131415161718191A36
:1002A0001B1C1D2F3130354C2223252628292A2CB2
:1002B0002D2F3032333536383A3B3D3E40424345B0
:1002C00047494A4C4E5051535557595A5C5E6062EB
:1002D000646668696B6D6F71737577797B7D7F81FB
:1002E000838587898A8C8E90929496989A9C9E9FFB
:1002F000A1A3A5A7A8AAACAEAFB1B3B4B6B8B9BB19
:10030000BCBEBFC1C2C3C5C6C7C9CACBCCCDCED087
:10031000D1D2D2D3D4D5D6D7D7D8D9D9DADADBDB74
:10032000DBDCDCDCDCDCDDDDDDDDDCDCDCDCDCDB0B
:10033000DBDBDADAD9D9D8D7D7D6D5D4D3D2D2D154
:10034000D0CECDCCCBCAC9C7C6C5C3C2C1BFBEBC47
:10035000BBB9B8B6B4B3B1AFAEACAAA8A7A5A3A1B8
:100360009F9E9C9A98969492908E8C8A898785837A
:10037000817F7D7B79777573716F6D6B696866645A
:1003800062605E5C5A5957555351504E4C4A49472A
:10039000454342403E3D3B3A3836353332302F2DCF
:1003A0002C2A292826252322FFAA7F554000010157
:1003B0000101010101010102020202020202020224
:1003C00003030303030303030404040404040405F4
:1003D00005050505060606060607070707070808B8
:1003E0000808090909090A0A0A0B0B0B0C0C0C0D69
:1003F0000D0D0E0E0E0F0F0F101011111112121302
:10040000131414151516161717181819191A1A1B7C
:100410001B1C1D1D1E1E1F202021222223242425DB
:100420002626272829292A2B2C2D2D2E2F30313214
:1004300032333435363738393A3B3C3D3E3F404124
:1004400042434445464748494A4C4D4E4F5051530C
:1004500054555658595A5B5D5E5F616264656668C3
:10046000696B6C6D6F7072737577787A7B7D7E8047
:1004700082838587888A8C8E8F91939596989A9C93
:100480009EA0A2A3A5A7A9ABADAFB1B3B5B7BABCA7
:10049000BEC0C2C4C6C9CBCDCFD1D4D6D8DBDDDF78
:1004A000E2E4E7E9EBEEF0F3F5F8FAFDFF1E0F05E5
:1004B0007F3F1F643214643214783C1E1E140A05F8
:1004C0002B4414001A000900130005002921040020
:1004D0001500160017000A001A7C1D001B000600FC
:1004E0000700190000000000000081522C00407E2F
:1004F0002A2433001C0018000F000D0034311200B4
:100500000C000800110010001B7C3800370036007A
:100510000B000E00000000000000025228432934A6
:100520002B441E021F0220022102220229212252F4
:100530000000000027000000E100000000000000B3
:100540000000000000000000000001520052407E48
:100550002A24270226022502240223023500310024
:1005600030002F002E002D003502310230022F0204
:100570002E022D02000000000000035228432934FF
:100580002B443A003B003C003D003E0029213F0047
:1005900040004100420043001A7C000000004C0073
:1005A0004400450000000000000004520052407E5C
:1005B0002A24270026002500240023022E002D00D7
:1005C00023002200210036002502380020001F00F1
:1005D0001E003700000000000000035228432934A9
:1005E000A800AC00AB00AA00A900AE0029210000C1
:1005F0000000D300D100D200E100000000000000A4
:100600000000000000000000000004520052E3005F
:10061000DD0000000000DC00D000CE00DE000000A5
:100620000000DA00D9000000DF0000000000DB005D
:10063000CF00CD000000000000000000000000001E
:1006400020782C782B7828782778307846002D78F9
:100650002E78247823783478E10032782F78267841
:100660002578317800000000000000000052E3000F
:10067000005200004A004B004F00510000000000F3
:100680000000000000000000000000004D004E00CF
:100690005000520000000000000003522800E30058
:1006A000200011241FBECFEFDAE0DEBFCDBF04B6BD
:1006B00003FE18C08091BF049091C004A091C104B2
:1006C000B091C2048730904BA740B04B59F41092C0
:1006D000BF041092C0041092C1041092C204E0E062
:1006E000F8E3099524E0ACEDB1E001C01D92AF3B09
:1006F000B207E1F711E0A0E0B1E0E0E3FFE502C0FE
:1007000005900D92AC3DB107D9F70E94A3240C943B
:10071000272F0C9400009C01FB019A9581159F41A5
:1007200030F4832F817031FD82600995089580E057
:10073000FCCF909373048093720408959093750492
:1007400080937404089521E030E002C0220F331F2B
:100750008A95E2F78091740490917504822B932B13
:100760000E949E03089521E030E002C0220F331F53
:100770008A95E2F7209530958091740490917504E4
:10078000822393230E949E030895983098F5863023
:1007900088F5E82FF0E086E0989FE00DF11D112428
:1007A0008E2F877041E001C0440F8A95EAF783E0FD
:1007B000F695E7958A95E1F7EE0FFF1FEE0FFF1F05
:1007C000EB5CFB4F20E030E070E05191DF011197CE
:1007D000CB01022E02C0969587950A94E2F78170AC
:1007E00081958527842385278C932F5F3F4F243065
:1007F000310559F70895983078F5863068F5E82F77
:10080000F0E086E0989FE00DF11D11249E2F977077
:1008100083E0F695E7958A95E1F7EE0FFF1FEE0F5F
:10082000FF1FEB5CFB4F40E050E080E0219130E0A7
:10083000092E02C0369527950A94E2F721703327D6
:10084000042E01C0220F0A94EAF7822B4F5F5F4FFC
:100850004430510559F7089580E0089580917D0452
:1008600090917C04981301C008958F5F8770FACF30
:10087000E0EEF1E09191891303C0DF0111971C9222
:1008800091E0E63EF907B1F70895909177048095DD
:10089000892380937704282F2770211111C089178D
:1008A00079F09091BE0492FF0BC08695869586954F
:1008B0000E94B30310927704109279041092780486
:1008C0000895982F909580917004892380937004E7
:1008D000089580916F04811531F010926F04109289
:1008E0007B0410927A0408957830B8F46630A8F446
:1008F0008530B0F4E62FF0E096E0799FE00DF11D31
:10090000112490E3899FE00DF11D1124EE0FFF1FCC
:10091000E054FB4F85919491089580E090E0089514
:1009200081E0FCCF803E9105D9F1C8F48133910577
:1009300009F482C048F48932910509F472C08A3200
:10094000910509F480C0089589339105E9F0823852
:100950009105D1F08533910509F45EC00895843E78
:100960009105D9F148F4823E910539F1833E910514
:1009700049F181EE90E00895863E9105C9F1873EE8
:10098000910509F43EC008952091BD042370211102
:1009900064C02091BE0423FF14C089E290E0089552
:1009A0002091BD0420FD45C03091BE0430FF09C038
:1009B00024FD24C083EE90E008952091BD0422FD23
:1009C000F7CF08952091BD0422FD44C03091BE04AC
:1009D00030FD43C024FFF5CF11C02091BE0421FF9C
:1009E000F0CF8091BD0484FD09C087EE90E00895AA
:1009F0002091BD0423FFE5CF24FFF7CF80E090E0F6
:100A000008952091BD0423FD2BC03091BE0431FF19
:100A1000E1CF84EE90E008952091BD0425FFD1CF71
:100A2000BCCF2091BD0425FD1EC02091BE0423FF34
:100A3000C8CF89E390E008952091BD0426FFC1CF7F
:100A40008AE290E008952091BD0426FFBACF81E3A9
:100A500090E0089582EE90E0089580EE90E0089591
:100A600086EE90E0089585E390E008959091BD04AE
:100A700092FF06C0282F28712830F9F4877F846000
:100A800093FF06C0282F28712831F1F4877E8461F6
:100A90002091BE0420FF06C0382F38713830D9F4B9
:100AA000877F816021FF06C0282F28712831D1F46B
:100AB000877E816194FD877E0895282F24712430DC
:100AC000F9F68B7F8860DCCF282F2471243101F761
:100AD0008B7E8861DDCF382F3171313019F78E7FF1
:100AE0008860E0CF282F2171213121F78E7E886127
:100AF000E1CF1F93CF93DF930E949204EC01811505
:100B000022E5920708F05DC0811540E5940708F0E2
:100B1000DBC0803E910528F58D3C910508F0ACC006
:100B2000883A910578F4853A910508F0A2C08130A1
:100B3000910509F441C00497813A9105E8F1C0E0BC
:100B4000D0E03AC0885A91094B97C8F7C85AD0E00C
:100B5000CC0FDD1FCA55DE4F0990D881C02DD4645B
:100B60002BC0811550E49507F8F4C11580E2D80731
:100B700008F0C3C0C83ED105F8F0CE019A958115A2
:100B80009F41E8F68D2F0E943605182FCE01992738
:100B90000E949204212F30E0322F2227E901CC2736
:100BA000DF71C82BD92B08C099270E949204CC274B
:100BB000DF70C82BD92BD06ACE01DF91CF911F9166
:100BC0000895803842E59407C8F5803652E59507C8
:100BD00008F05BC0C03482E5D807D0F4C03292E59B
:100BE000D90708F04BC08C2F8695869520E2829F0E
:100BF000C0011124C37021E030E0A90102C0440FFC
:100C0000551FCA95E2F7EA01C82BD92BDD68D4CF6E
:100C10008C2F86958695877050E2859FC0011124A0
:100C2000C37021E030E0A90102C0440F551FCA95EE
:100C3000E2F7EA01C82BD92BDC68BECF803C52E535
:100C4000950758F48F71C03AD245A0F590E0982FDF
:100C50008827EC01C46FD06AAFCF805C9245809743
:100C600008F06DCFDC2FCC27CC27DF71C06FD06AA6
:100C7000A3CFA497D064A0CFD0659ECFCF71D0E092
:100C8000DC2FCC27C16FD06A97CF86958695877069
:100C900020E2829FC0011124C37021E030E0A9014D
:100CA00002C0440F551FCA95E2F7EA01C82BD92BA1
:100CB000DA6882CF0E943605C82FD0E0DC2FCC271F
:100CC000CC27DF71D06278CF8F710E94360565E046
:100CD000D695C7956A95E1F7CF70D0E0DC2FCC2789
:100CE000282F30E084FF05C054E0220F331F5A95AF
:100CF000E1F7C22BD32BD0695FCF8D2F8F710E946C
:100D00003605182FCE0199270E949204212F30E03A
:100D1000322F222722273F71282B392BE901D2CFEE
:100D2000A0E0B0E0E6E9F6E00C94322D8C01E09012
:100D30007404F09075048091720490917304E82A11
:100D4000F92ACFE0D0E0CC24C394D12CC6010C2EDC
:100D500002C0880F991F0A94E2F78E219F21892BE8
:100D600049F4219798F7B12C8B2DCDB7DEB7E9E088
:100D70000C944E2DBC2EB8018C2F0E9474040E943E
:100D80007905019771F3F0CF0F931F93CF93FC0177
:100D9000858100811181811591F0611581F0C80173
:100DA0000E949006C82F682FC8010E94C503B80191
:100DB0008C2F0E947404CF911F910F910895C80148
:100DC0000E94FB03C82FF3CFCF93DF93D82FC92FF7
:100DD0000E9490066D2F7C2F0E9474040E9479055A
:100DE000DF91CF910895FC0184818115A1F080816C
:100DF00091810E94E406282F92959F70963099F079
:100E000060F4925F9F70923030F4203F89F038F4A4
:100E100081E0283E38F080E008959A5FF3CF81E0CA
:100E2000243FC9F7089581E0283E20F0213FF9CF03
:100E300081E00895089580E00895F894E82FE29500
:100E4000EF70F0E041A18F7021E030E0B90102C005
:100E5000660F771F8A95E2F7CB01962F9095942322
:100E600091A392A1892B82A37894089508958091EB
:100E70004F0480FD14C081FD14C082FD16C0809116
:100E80004E04811581F08E3180F420E5829FC001EF
:100E900011246EE170E00E948E2D862F089584E16A
:100EA000089588E2089588E0089580E50895809186
:100EB0004F0480FD17C081FD17C082FD19C08091CD
:100EC0004D04811599F0883298F428E0829FC00182
:100ED000112468E270E00E948E2D6115710551F0B9
:100EE000862F089562E0FCCF64E0FACF61E0F8CF8E
:100EF00068E0F6CF81E00895A0E0B0E0E2E8F7E036
:100F00000C94322D8901E42FF0E0E355FC4F611180
:100F10000FC0E491BE2E2E2FD80111962C9311975D
:100F2000EC931296BC92CDB7DEB7E9E00C944E2D4F
:100F3000C82FD0E0E62EF12C3491232F86E08C9F31
:100F400060018D9FD00C1124EFEFF0E0C601BF01CE
:100F50000E947A2DCC0FDD1F45E5469FC001479FBB
:100F6000900D1124C81BD90BAC2FAA0FAC0FAF01E9
:100F70004E195F09349FC001359F900D1124B92E81
:100F8000AE9DE001AF9DD00D1124CD2FDD27AF0127
:100F90004C1B5D0BEA013C9FA0013D9F500D1124AD
:100FA000EF01CA1BD109DE01AE9DE001AF9DD00D5E
:100FB000BE9DD00D1124CD2FDD27EC1BFD0B3E9FD8
:100FC000D0013F9FB00D1124EB2F63307105D1F09C
:100FD000DCEFCD16D3E0DD0658F461307105B1F0D9
:100FE0006230710509F098CFE32F292FBB2E94CFE3
:100FF0006430710571F06630710509F48DCFE92F09
:10100000B52E8ACF292FB32EE52F86CFE32F252F9C
:1010100083CFE92FB32E2B2F7FCF809167048230AF
:1010200060F4817082608093670480916A048138E3
:1010300018F080E880936A0408958235B0F38170D7
:101040008065F1CFE4E6F4E01182828184608283DE
:101050000895FA01811511F009950895FB01FCCF5F
:10106000FC01680F791F8FEF41E39191892728E0F8
:1010700030E0982F990F87FF09C0892F84272150CE
:101080003040B9F7E617F70781F70895892FF7CFB2
:10109000A3E0B0E0EEE4F8E00C94392D9C018091DF
:1010A0000A0290910B0282179307A1F030930B0272
:1010B00020930A02E0912B04F0912C04309751F018
:1010C00083E089833B832A830680F781E02DCE016C
:1010D000019609952396E2E00C94552DA3E0B0E02B
:1010E000E4E7F8E00C94392D9C018091080290917E
:1010F000090282179307A1F0309309022093080296
:10110000E0912B04F0912C04309751F084E0898316
:101110003B832A830680F781E02DCE010196099555
:101120002396E2E00C94552D9C01FC0132968FEF42
:1011300090E04191461751F08F3F19F4411101C0E1
:10114000892F9F5F9630A9F78F3F09F40895280FE4
:10115000311D87FD3A95F901628308952FB7F89400
:101160008091090490910A04A0910B04B0910C04A1
:101170002FBF0895962F2091BE0422FF10C0682F24
:10118000660F660F660F692B609377040E94A303B6
:101190000E94AE08909379048093780408950E9489
:1011A000A303089590916F04292F2823211561F03E
:1011B0008095892380936F04811539F00E94AE08D1
:1011C00080937A0490937B04089580E090E0F8CFB8
:1011D0000E94AE082091520430915304232B211514
:1011E00021F08093EE039093EF032091540430910B
:1011F0005504232B211521F08093EC039093ED03EC
:10120000E0912B04F0912C04309749F082E0809318
:1012100050040480F581E02D80E594E0099508955F
:10122000611509F44BC0E3E3E80FE33150F4F0E05B
:10123000E75DF04D0C94A22D0E94370781958093B5
:1012400053040E94E80808950E943707F8CF0E94CF
:101250003707819580935204F4CF0E943707FACF65
:101260000E94570780935404ECCF0E945707819542
:10127000F9CF0E945707819580935504E2CF0E94D1
:101280005707FACF815D990B21E030E001C0220FB2
:101290008A95EAF780915104822B80935104D1CF33
:1012A00080914F04816080934F04CBCF80914F0495
:1012B0008260F9CF80914F048460F5CF4091520451
:1012C0008D3C59F48091530487FF0DC01092530454
:1012D000411559F410924E0408C08E3C81F480915F
:1012E000530418169CF3411581F080915404909199
:1012F0005504892B8111A5CF10924D04A2CF8F3CAC
:1013000041F447FFF0CF10925204809153048115AD
:10131000E0CF803D19F41416B4F3E5CF9091540456
:10132000893D29F41916FCF610925404DCCF8A3D4D
:1013300019F497FFD8CFF8CF909155048B3D29F43D
:1013400097FFD1CF10925504CECF8C3D19F41916CA
:10135000CCF3C9CF9FE2980F983090F4815D990B40
:1013600021E030E0B90102C0660F771F8A95E2F7ED
:10137000CB01809590915104892380935104B3CF80
:101380008D3D31F480914F048E7F80934F04ABCF1D
:101390008E3D21F480914F048D7FF7CF8F3D09F072
:1013A000A2CF80914F048B7FF0CF2FB7F89460913C
:1013B000090470910A0480910B0490910C042FBFD2
:1013C00008959C014FB7F8948091090490910A0404
:1013D000A0910B04B0910C044FBF821B930B089596
:1013E000809107020895FC019B018091FD0190917D
:1013F000FE018617970740F0672B29F48091E800DB
:101400008E778093E800C90140E0009741F44111D4
:1014100006C08091E80082FF2FC080E008952091EF
:1014200023042115A9F12530A9F12091E80023FD1D
:101430002DC02091E80022FDECCF2091E80020FF94
:10144000E4CF3091F3002091F200009719F028309A
:10145000310558F041E02830310509F040E0209195
:10146000E8002E772093E800D0CF41914093F1001F
:1014700001972F5F3F4FE9CF80912304811541F001
:10148000853041F08091E80083FFC3CF81E008956B
:1014900082E0089583E008958091F70187FF13C0EB
:1014A0008091E80082FF06C08091E8008B778093EE
:1014B000E8000895809123048111F2CF089580916E
:1014C00023048115D9F38091E80080FFF8CF809143
:1014D000E8008E77ECCF2091E4003091E50095E6AE
:1014E000A9018091EC008170811531F08091E800B4
:1014F00080FF06C080E008952091E80022FD1AC018
:1015000080912304811589F0853089F08091EB006A
:1015100085FD0FC02091E4003091E500421753078C
:1015200001F39A95E9F684E0089582E0089583E056
:10153000089581E00895E8EDF0E080818E7F80835A
:101540001092E2001092DA001092E100A0EEB0E0FA
:101550008C9181608C9380818F77808319BCA7EDFB
:10156000B0E08C918E7F8C9380818F7E80831092EF
:10157000F6010895982F9093E900242F762F50E0DC
:10158000981731F07091EC002091ED005091F0002F
:1015900021FD06C09F5F973071F78093E9000895A1
:1015A0003091EB003E7F3093EB003091ED003D7FBA
:1015B0003093ED003091EB0031603093EB0070938D
:1015C000EC002093ED005093F0002091EE0027FDF9
:1015D000E1CF0895A0E0B0E0E0EFFAE00C94332D05
:1015E000C8EDD0E088818F7E8883E7EDF0E08081D0
:1015F0008160808384E082BF81E08093F6018881EE
:101600008E7F888302EE10E0F80110821092DA00DB
:1016100081EEC82ED12CF601108288818F778883C5
:1016200088818068888388818F7D888319BC109227
:1016300023041092F5011092CB031092F40190EE66
:10164000E92EF12CF70180818B7F80838881816076
:10165000888342E060E080E00E94BA0AF60180815F
:101660008E7F8083F80180818160808380818860A3
:101670008083F70180818E7F808388818061888369
:10168000CDB7DEB7E8E00C944F2DE0917D0490914A
:101690007C0427E0E91302C080E00895AE2FB0E09B
:1016A0002E9FF0011124E258FB4F3181361306C002
:1016B0003081381303C03581341304C0FD013196E5
:1016C000E770E8CF81E0089580912404811110C073
:1016D0008091D80080618093D8008AE18A95F1F7E3
:1016E00000C08091D90080FF0AC081E0809324046B
:1016F00081E090912404913009F080E0089582E027
:10170000809324040E949B0A10922304F1CF0F932C
:101710001F930E94640B811529F00E94D5091F9127
:101720000F9108950E94D509009125041091260477
:101730002091270430912804600F711F821F931F8E
:10174000EECF0E94870B08950E94640B811519F05B
:101750000E94AE0808950E94870BCB0108950E9455
:10176000640B811559F0E0912B04F0912C04309713
:1017700029F00190F081E02D0995089580E0089509
:10178000409114018091670480FF24C020911301CF
:1017900030E0C901880F991F820F931F845E9C4F10
:1017A000539A6BB1677F7BB17860EFB7F89450E0E4
:1017B0009A01220F331F240F351F280F391F2817B6
:1017C0003907E9F4EFBF8FE594E00197F1F700C026
:1017D000000008958091150190911601282F30E0A6
:1017E000F901EE0FFF1FE20FF31FE45EFC4F8917B4
:1017F00068F61182108212828F5F3396F8CFDC0177
:101800004D91CD0158E07BB9000000C047FF6BB996
:10181000440F000000C000C000C06BB900C05A9562
:1018200091F7CDCFEF92FF921F93CF93DF93EC010F
:1018300010E0EE24EA94F12C60911701161770F075
:101840000E94C00B9A818C8190FF28C08F5F8C838F
:10185000DF91CF911F91FF90EF9008958091150136
:10186000810F9927991F9C01220F331F280F391FC1
:10187000245E3C4F40916A04413808F040E870E033
:10188000C7010E948E2D962F8C8160916904199F4B
:10189000800D11240E947C071F5FCECF8150D7CFCF
:1018A000A0E0B0E0E6E5FCE00C94302DEC018A818C
:1018B000BB24B39480FF02C0BB24BA948C81A09057
:1018C0001701811109C091E0B91202C08FEF8A0D92
:1018D00080931B0381E08C83E12CF12CEA14B8F097
:1018E0000E94C00B90911B03E1E0BE1255C0809195
:1018F00017018150911519F08FEF890F91E08093B6
:101900001B039C83CDB7DEB7EBE00C944C2D80918C
:1019100015018E0D9F2D911D8C01000F111F080FB9
:10192000191F045E1C4FF80111821082128234E0EC
:10193000C32ED12C912C80911B03890D873344F148
:1019400066E30E946C2D892F082E001C00088E155E
:101950000F04A9F480916A048C9DA0018D9D500D07
:1019600011245595479555954795413808F040E81D
:10197000980160916904809168040E947C079B0C27
:10198000F1E0CF1AD108B9F68FEFE81AF80AA6CF1E
:1019900087FFDACF8A0DD8CF892F90E0019660912A
:1019A000170170E00E948E2D982FA9CF0F931F93DF
:1019B000CF93DF93EC018C81811109C081E08C838E
:1019C00010921A0392E09093070180930601109100
:1019D000150120911601812F90E0FC01EE0FFF1FF1
:1019E000E80FF91FE45EFC4F821750F100E06091B0
:1019F0001701061758F10E94C00B809106019091C3
:101A00001A03980F90931A0320910701280F20932F
:101A10000701121654F4209117012150330B092E9F
:101A2000001C00089217030634F08195809306018C
:101A3000813009F41C82DF91CF911F910F9108959D
:101A40001182108212828F5F3396CECF202F30E02A
:101A500070E0C9010E948E2D810F90E040911A0321
:101A6000FC01EE0FFF1FE80FF91F042E001C0008F9
:101A700024173005C4F040910701042E001C000813
:101A80004217030684F09F01245E3C4F40916A0494
:101A9000413808F040E860916904809168040E9430
:101AA0007C070F5FA4CFE45EFC4F1182108212828C
:101AB000F8CFA6E0B0E0EFE5FDE00C94332D8D8388
:101AC0009E83AD81BE811496FC912F2F30E0D90109
:101AD0000E94182F9B01AC010E94E32E6B017C0138
:101AE00080E290E09C012F1B3109F901A5E5B0E0EF
:101AF000A70196010E94E32E69837A838B839C83DE
:101B00009F01DF010E94A82D9B01AC010E94EE2ED7
:101B10009B01AC012C0D3D1D4E1D5F1D69817A811D
:101B20008B819C810E94F62E022F30E00A3248F50C
:101B3000C901880F991F820F931F95958795F82EDD
:101B4000F09410E085E5E82EE01A8091170118174F
:101B500038F10E94C00BAD81BE8114969C9181E04A
:101B6000911519F0903219F48FEF8093050180914F
:101B70000501890FED81FE8184832696E8E00C94AF
:101B80004F2D85E590E0AC01421B530B9A01CA0131
:101B9000880F991F820F931F97FFCFCF0196CDCF4C
:101BA0008E2D11FD802F40911501410F5527551F96
:101BB0009A01220F331F240F351F245E3C4F4F2DF7
:101BC00051E8F51608F040E8609169040E947C072E
:101BD0001F5FBBCF9091670490FF11C090911501DA
:101BE00050911601292F30E0F901EE0FFF1FE20F8F
:101BF000F31FE45EFC4F951718F00E94C00B089588
:101C00008183608342839F5F3396F5CFA3E0B0E08A
:101C1000ECE0FEE00C94392D9091670490FF0DC02C
:101C2000413808F040E89E012F5F3F4F0E947C073B
:101C30004B8169818A810E94EA0D2396E2E00C942F
:101C4000552DCF93DF93EC01EC81F0E0E855FD4F8B
:101C50004491E7E6F4E0628181810E94060E8C8166
:101C60008F5F8C83DF91CF910895CF93DF93EC0149
:101C7000E7E6F4E0438162818C810E94060E8C814C
:101C80008F5F8C83DF91CF91089581E08093E00096
:101C900080E28093D8001092C9008FE19EE4019702
:101CA000F1F700C0000087E090EBDC018093BF04F7
:101CB0009093C004A093C104B093C20488E19CE057
:101CC0000FB6F894A895809360000FBE90936000C3
:101CD000FFCF0F931F93CF93DF938B01EA01909176
:101CE0002304943059F58093E9008FEF9091E80038
:101CF00095FD06C095ED9A95F1F700008A95B1F72C
:101D00008091E80085FF1AC00E946B0A811111C002
:101D10008091E80085FD06C08091E8008E77809371
:101D2000E800F2CFF80181918F018093F1002197B3
:101D300079F78091E8008E778093E800DF91CF916A
:101D40001F910F910895CF93DF93D82FC92F48E0AB
:101D500050E0682F792F81E00E94690E88E0ED2F16
:101D6000FC2FAFEFB1E001900D928A95E1F7DF9182
:101D7000CF910895BC0146E050E082E00E94690ED8
:101D80000895BC0143E050E082E00E94690E08958E
:101D9000A0E0B0E0EEECFEE00C94312DF82EE92E40
:101DA000B62EA72E8A018091F001CC24C394D12CA9
:101DB0008A3018F48AE0C82ED12CC1E0D0E06B2D17
:101DC0007A2D8F2D9E2DF8010995811116C021962F
:101DD000CC16DD0694F0CC9FC001CD9F900D900DE8
:101DE000112420E030E045E34A95F1F700002F5F31
:101DF0003F4F28173907B9F7E2CFCDB7DEB7EAE092
:101E00000C944D2D9091BE0492FB222720F92817A7
:101E100079F080FB92F99093BE046091BD047091BB
:101E2000BE0484E090E00E94AE2E82E00E94450451
:101E3000089560915A048CE090E00E94902E0895DD
:101E40002091C803082E000C990B820F911D27FDCD
:101E50009A9563E070E00E948E2DE82F87FF02C004
:101E6000E3E0E80FE093C8030E2E000CFF0BEF56E3
:101E7000FE4F808180935A040E94190F089580912B
:101E8000700490917604892B8093DE0180916F0419
:101E9000811519F10E94AE0820917A0430917B04DB
:101EA000821B930B8838934110F00E946904809143
:101EB000DE0190916F04892B8093DE0120E080EE9B
:101EC00091E0FC013081019631112F5F31E0863EB7
:101ED0009307B9F721110E94690448E050E06DE2D0
:101EE00074E08EED91E00E94562E892BA9F088E0D7
:101EF000EEEDF1E0ADE2B4E001900D928A95E1F7EC
:101F0000E0912B04F0912C04309731F00280F381A2
:101F1000E02D8EED91E009950895811521F00E9444
:101F200061040E943F0F0895811541F080959091C2
:101F300076048923809376040E943F0F08958115CB
:101F400039F090917004892B809370040E943F0FA8
:101F50000895811539F090917604892B8093760449
:101F60000E943F0F0895CF93C82F8115A9F08CEFE1
:101F70008C0F813A98F4E0EEF1E08191C81709F4F2
:101F800040C021E0E63EF207C1F76C2F8EED91E0F4
:101F90000E9494080E943F0FCF91089580E28C0F19
:101FA000883068F4C77021E030E001C0220FCA9584
:101FB000EAF780917004822B80937004EBCF8BE55D
:101FC0008C0F833038F42C2F2452330BC9010E941C
:101FD0004808E2CFE8E5EC0FEB3150F4F0E0EE0F0B
:101FE000FF1FEA55FE4F808191810E946E08D4CF79
:101FF00083E38C0F833180F661E08C2F0E941009FF
:10200000CBCF8C2F0E9438040E943F0FBECF81158A
:1020100081F19CEF980F913A28F40E9438040E94B5
:102020003F0F089590E2980F983050F4877091E038
:1020300001C0990F8A95EAF7892F0E946104EFCFBA
:102040009BE5980F933028F480E090E00E944808C8
:10205000089598E5980F9B3128F480E090E00E9465
:102060006E08089593E3980F933118F460E00E948E
:1020700010090895EF92FF920F931F93CF93DF9370
:10208000EC018B017C0180EEE81AF1086FE97FE03A
:1020900098E0E916F10410F069EA7FE0CE010E94B1
:1020A0008B038C2F0E94B30F0115110599F48C2F0F
:1020B0000E9407106DE87FE098E0E916F10410F047
:1020C00064E97FE0CE010E948B03CDB7DEB7E6E086
:1020D0000C94512D8FE99FE00197F1F700C00000AB
:1020E00001501109E1CF0F931F93CF93C82F00E543
:1020F00010E0893311F000E010E08C2F0E94B30F44
:102100000115110539F48C2F0E940710CF911F91F2
:102110000F9108958FE99FE00197F1F700C000004B
:1021200001501109EDCFFF920F931F93CF93DF93CF
:10213000C62FD42F122F8115A9F0609362040E943C
:10214000AE089093F2018093F101C77081E001C065
:10215000880FCA95EAF70E949F0FCDB7DEB7E5E07A
:102160000C94522D80916204681334C08091F10167
:102170009091F2010E94E10920915F01309160018C
:102180008217930738F500E20D0FCD17A9F0C7703D
:10219000FF24F3948F2D01C0880FCA95EAF70E949F
:1021A0008D0F083048F48D2F877001C0FF0C8A9581
:1021B000EAF78F2D0E949F0F812F0E947310083025
:1021C00060F6D77081E001C0880FDA95EAF70E94C7
:1021D0008D0FC3CFC77081E001C0880FCA95EAF7A1
:1021E000F6CF811107C089EA611101C08AEA0E9415
:1021F000731008958130E9F78EE46111F8CF8BE414
:10220000F6CFA0E0B0E0E7E0F1E10C94342DE82F48
:10221000F0E0E85DFD4FD490282F26952695269571
:1022200030E0F901E85EFD4F0491877010E0082E60
:1022300002C0159507950A94E2F701701127F9017C
:10224000E85FFD4FE490F12C082E02C0F594E7946E
:102250000A94E2F791E0E922FF24F901E850FE4FE9
:10226000C491D0E002C0D595C7958A95E2F7C170B8
:10227000DD270115110519F081EE0E94B30FE1145D
:10228000F10419F086EE0E94B30F8D2D0E94731099
:10229000E114F10419F086EE0E94071001151105F2
:1022A00019F081EE0E940710CD2B19F08CE20E94EC
:1022B0007310CDB7DEB7E7E00C94502DCF9310929A
:1022C0007004C6E0E0EEF1E0DF018C2F1D928A95EC
:1022D000E9F780E090E00E94480880E090E00E94EA
:1022E0006E08109276040E943F0FE0E5F4E0DF01F3
:1022F0001D92CA95E9F710924E0410924D04109267
:102300004F040E94E808CF9108950E945E112FEFBC
:1023100084E39CE0215080409040E1F700C0000041
:1023200088E19CE00FB6F894A895809360000FBEFA
:1023300090936000FFCFAAE2B0E0E1EAF1E10C94F3
:10234000382D87EF91E0FC0101962091F100208368
:1023500021E08F3F9207B9F78091F801893009F4A5
:1023600056C0C8F4823009F4B2C0833009F481C089
:10237000813071F18091E80083FFE7C08091F7011F
:102380009091F8019A3008F0E0C0E92FF0E0E45CA9
:10239000F04D0C94A22D8A3009F488C08B3051F78F
:1023A0008091F701813231F78091FB019091FC011E
:1023B000892B01F78091E800877F8093E8000E94D5
:1023C0004C0A8091F901809304010E945E11D2CFE2
:1023D0008091F701813A71F68091E800877F8093C0
:1023E000E8008091FB019091FC01892B61F060E095
:1023F00080E090E070E00E94F3098091E8008B7724
:102400008093E800B7CF68E08FEF91E0F3CF809141
:10241000F701813209F0AECF8091FB019091FC0170
:10242000029708F0A7CF8091E800877F8093E800AB
:102430008091E80082FF18C09091F3008091F20033
:10244000029731F48091F100813011F0863021F44F
:102450008091F100809307028091E8008B77809350
:10246000E8000E944C0A86CF809123048111E0CFBE
:1024700081CF8091F701813A09F07CCF8091FB01F7
:102480009091FC01892B09F075CF8091E800877F3E
:102490008093E8008091E80080FFFCCF80910401E8
:1024A0008093F1008091E8008E77D9CF8091F70179
:1024B000813209F05FCF8091E800877F8093E80048
:1024C0000E944C0A8091FA018093F30153CF8091CE
:1024D000F701813A09F04ECF8091E800877F809321
:1024E000E8008091E80080FFFCCF8091F301D8CF15
:1024F000803889F0823849F58091FB018F708730F0
:1025000020F58093E9008091EB0085FB882780F916
:102510001092E90007C09091CB0391959270809141
:10252000F401892B9091E800977F9093E8008093C5
:10253000F1001092F1008091E8008E7723C08111A4
:1025400016C08091F901813011F18091E80083FF7C
:102550000AC08091E800877F8093E8008091EB00BB
:1025600080628093EB00AA96E3E00C94542D8230B5
:1025700061F78091F901811589F01092E90080914D
:10258000E800877F8093E8000E944C0ADECF81E05C
:10259000933009F080E08093CB03EFCF8091FB0173
:1025A0008F702FEF280F263080F68093E90020915E
:1025B000EB0020FFE2CF933031F48091EB0080629A
:1025C0008093EB00DACF9091EB0090619093EB0059
:1025D00021E030E0A90102C0440F551F8A95E2F7BF
:1025E0004093EA001092EA008091EB008860E8CF07
:1025F0008111ABCF1091F9011F778091E3008078B2
:10260000812B8093E3008091E800877F8093E8002E
:102610000E944C0A8091E80080FFFCCF8091E3008B
:1026200080688093E30083E0111101C082E0809311
:1026300023048BCF8058823008F087CF4091F90176
:102640005091FA014C3D83E0580799F583E08A8365
:102650008AE289834FB7F894DE01139620E03EE0CA
:1026600051E2E32FF0E050935700849120FF03C024
:1026700082958F703F5F8F708A30C8F0895C90E0E0
:102680008D939D932F5F243161F74FBF8091E800B8
:10269000877F8093E8006AE270E0CE0101960E9495
:1026A000F3098091E8008B778093E8004ECF805D3E
:1026B000E6CF2091FB013091FC01852F99278330D3
:1026C000910509F160F48130910509F472C0029717
:1026D00009F03BCF8BE390E0E7E6F1E029C08132DF
:1026E000910509F45AC0829709F02FCF21153105C1
:1026F00009F469C02130310509F027CF8BE790E05C
:10270000ECEAF0E015C0CA0199274130B1F18230FE
:10271000910509F43AC0892B09F017CFE4EFF1E0F5
:10272000E4918E2F90E0E4EFF1E0009709F40DCFF3
:102730002091E800277F2093E8002091FD0130914F
:10274000FE018217930708F49C0140E02115310532
:1027500009F03EC041113CC08091E80082FDA1CF4C
:1027600080912304811509F49CCF853009F499CF19
:102770008091E80083FFF0CF94CFEAEDF1E0E4919F
:102780008E2F90E0EAEDF1E0D0CFE4EBF1E0E491C0
:102790008E2F90E0E4EBF1E0C8CF2115310571F008
:1027A0002130310509F0D1CE89E090E0E2E9F1E095
:1027B000BFCF82E190E0E2EAF1E0BACF89E090E0B9
:1027C000E9E7F1E0B5CF80E490E0E7E2F1E0B0CFF7
:1027D00080912304811509F464CF853009F461CF19
:1027E0008091E80083FD5DCF8091E80082FDB4CF49
:1027F0008091E80080FFAACF9091F3008091F200D1
:102800002115310519F08830910550F041E0089705
:1028100009F040E08091E8008E778093E80096CF41
:1028200044914093F1003196215031090196E8CF4F
:10283000803809F08ACE8091E800877F8093E80095
:102840008091F5018093F10076CE81117ECE1091BA
:10285000F901123008F079CE8091E800877F8093EB
:10286000E8001093F5010E944C0A111581F084E0F4
:102870008093230442E061EC81E00E94BA0A42E2C4
:1028800061EC82E00E94BA0A809123045ECE8091BE
:10289000E30087FDECCF81E0EBCFA0E0B0E0E3E523
:1028A000F4E10C94332D8901D42FC52F6B017C01E9
:1028B0000E940D08A8016D2F7C2F88E090E00E94F7
:1028C000A22E98014D2F5C2FB601C70100E20E9495
:1028D000D22D622F84E290E00E94902ECDB7DEB719
:1028E000E8E00C944F2DE7E6F4E083E0808311826A
:1028F0008FEF828380E883831482A4E6B4E012968B
:102900008C911297836012968C93758123E030E04E
:102910004FEF50E860E0868197810E944D14089542
:1029200080916B04833018F48F5F80936B04209147
:102930006704309168044091690450916A04609181
:102940006B0470916C0480916D0490916E040E94F0
:102950004D14089580916B04811519F08150809376
:102960006B04209167043091680440916904509190
:102970006A0460916B0470916C0480916D04909175
:102980006E040E944D140895A3E0B0E0EAECF4E177
:102990000C94312DE82ED62EF42EB22E9091670491
:1029A00090FF45C030916804381308C080916904D5
:1029B000861304C080916A04841729F0809166040C
:1029C000826080936604E92FE695AE2FB0E0A859A7
:1029D000BE4F8C91809364049E7F923061F54F2DA1
:1029E00081E8F81608F040E89E012F5F3F4F6D2DFB
:1029F0008E2D0E947C074B8169818A810E94EA0D9D
:102A00003E2D30936804D0926904F0926A04B114A8
:102A100071F02091670460916B0470916C044D2DEE
:102A20005F2D80916D0490916E040E944D14239649
:102A3000EAE00C944D2D823019F4F0906A04E0CF56
:102A40008630F9F28930E9F28931D1F6E9519E2FC9
:102A50009170A92EE695F0E0E855FC4FE491C12C69
:102A60000E2F10E060911701C61618F00E94C00BDF
:102A7000C7CF2C2D30E0C09EC001C19E900D112407
:102A800070E00E947A2D8E2DA11017C0860F9091B4
:102A90001501A901490F511D9A01220F331F240F5F
:102AA000351F245E3C4F4F2D91E8F91608F040E8A1
:102AB0006D2D0E947C07C394D5CF861BE8CFE7E637
:102AC000F4E0818121E043816281885F0E94C41427
:102AD0000895E7E6F4E0818121E043816281885036
:102AE0000E94C4140895E7E6F4E0628121E1620FD8
:102AF00008F46FEF21E0438181810E94C41408959E
:102B0000E7E6F4E0628121E1621B08F460E021E085
:102B1000438181810E94C4140895E7E6F4E0438173
:102B200021E1420F08F44FEF21E0628181810E9490
:102B3000C4140895E7E6F4E0438121E1421B08F460
:102B400040E021E0628181810E94C4140895A8E0E0
:102B5000B0E0EDEAF5E10C94392D66EE7EEF80E011
:102B600090E00E94AE2E60E082E090E00E94902E05
:102B700060E083E090E00E94902E10927304109227
:102B8000720460E074E184E090E00E94AE2E60E0A8
:102B900086E090E00E94902E6FEF87E090E00E9428
:102BA000902E40E050E0BA0188E090E00E94A22E12
:102BB00060E084E290E00E94902E60E087E190E087
:102BC0000E94902E60E08CE090E00E94902E60E0E9
:102BD0008DE090E00E94902E19821A821B821C8246
:102BE0001D821E821F82188648E050E068E170E076
:102BF000CE0101960E94802E40E050E0BA0180E2B2
:102C000090E00E94A22E40E050E0BA018FE090E0F8
:102C10000E94A22E40E050E0BA0183E190E00E94C1
:102C2000A22E2896E2E00C94552DA1E0B0E0EBE155
:102C3000F6E10C942B2D462E4A01522EC32E37015D
:102C4000A82E880FBB08C5010E94B52CD82E81156F
:102C500009F475C0C50133E0880F991F3A95E1F773
:102C6000FC01E35DFE4F2381422F50E0211511F05E
:102C700041E050E0835D9E4FFC0164817581635F9C
:102C80007B4FCE0101960E94632EF4014081518159
:102C9000628173812FB7F8948091090490910A049E
:102CA000A0910B04B0910C042FBF841B950BA60BB5
:102CB000B70B84369105A105B10538F4B301C801FD
:102CC0000E94300899818917D1F1E42C042C000C62
:102CD000FF08C7010E94B52CD82E811106C0D12C47
:102CE0008D2D2196E0E10C94472DC70123E0880F3C
:102CF000991F2A95E1F7FC01E35DFE4F2381422FE6
:102D000050E06216710408F4A301835D9E4FFC013C
:102D100064817581635F7B4F852D9C2D0E94632E9E
:102D2000B301C8010E94300899818913D8CF0E944D
:102D3000D509F4016083718382839383D1CFA3018A
:102D4000B801852D9C2D0E94632ECACFA4E0B0E06F
:102D5000ECEAF6E10C94332D6B0184E0E82EF12CC3
:102D60000EE014E09E012F5F3F4F45E054E061E02C
:102D700080E00E941516811561F049815A816B81AE
:102D80007C81409301045093020460930304709388
:102D90000404409101045091020460910304709175
:102DA0000404F60140835183628373832496E8E030
:102DB0000C944F2DA1E0B0E0E0EEF6E10C94322D42
:102DC000EE24E394F12C03E114E09E012F5F3F4FCA
:102DD0004DEF53E063E082E00E941516082F811545
:102DE00039F1D12C80E01DC0C090FC03CD0C2C2DFE
:102DF00030E0A90146505C4F7A01E1E0F0E0EC0FD1
:102E0000FD1FED0DF11D1081FA019081191BB12EEE
:102E10001B149CF0912F17FD90E0191B111118C085
:102E2000D3949091F903D916F8F281110E94A10B65
:102E3000802F2196E9E00C944E2DBA94F701808101
:102E40008F5F808360E08C2D0E94F110802FE0CF97
:102E50001F5FF70180818150808361E08C2D0E948B
:102E6000F110802FDBCFA4E0B0E0E9E3F7E10C94B0
:102E7000382D4091F5035091F6036091F70370915E
:102E8000F8032FB7F8948091090490910A04A09157
:102E90000B04B0910C042FBF841B950BA60BB70B32
:102EA00011E084369105A105B10578F10E94870BE8
:102EB000DC01CB010296A11DB11D89839A83AB83EE
:102EC000BC8380914E0190914F01835F9B4F209175
:102ED0004D01422F50E0253010F044E050E0BE019B
:102EE0006F5F7F4F0E94632E84E090E00E94B52CBC
:102EF000182F811551F00E94D5096093F503709346
:102F0000F6038093F7039093F803812F2496E3E070
:102F10000C94542DCF92DF92EF92FF92CF93DF93D8
:102F2000CDB7DEB72B970FB6F894DEBF0FBECDBF7F
:102F300088E0E7E6F4E09E012F5F3F4FD901019062
:102F40000D928A95E1F74091640490916504809117
:102F5000660449879A878B87C090F103D090F2036B
:102F6000E090F303F090F4039FB7F89440910904C4
:102F700050910A0460910B0470910C049FBF4C198E
:102F80005D096E097F09E22F44365105610571051F
:102F900010F4811511F18091560190915701835FD2
:102FA0009B4F20915501422F50E02C3010F04BE008
:102FB00050E06E2F732F0E94632E85E090E00E94F8
:102FC000B52C811569F00E94D5096093F1037093C7
:102FD000F2038093F3039093F4031092660481E06C
:102FE0002B960FB6F894DEBF0FBECDBFDF91CF9109
:102FF000FF90EF90DF90CF900895A0E0B0E0E3E085
:10300000F8E10C942B2DFC016280448081E08483E4
:10301000E8EAF2E07490E7E2F3E0E491C0916A0438
:10302000C695C158D0E0CC0FDD1FED2EFF24812CBA
:1030300075E0972EAA24AA94B12C55245A94E71926
:10304000CE2ED12C80911701881638F00E94C00B2B
:10305000CDB7DEB7E0E10C94472D082D10E083E0FA
:10306000681668F4909EF001919EF00D1124E45FC3
:10307000FD4F8091680480838091690481834110B1
:103080002DC0909EF001919EF00D1124E45FFD4F44
:103090001382128280911501800F912F911D9C0146
:1030A000220F331F280F391F245E3C4F909EF001E2
:1030B000919EF00D1124E45FFD4F4281413808F0EC
:1030C00040E8909EF001919EF00D1124E45FFD4FC9
:1030D000618180810E947C078394B4CF909EE0013F
:1030E000919ED00D1124C45FDD4F8B818115E9F0D5
:1030F00081508B83589EC00111246C8170E00E9426
:103100007A2DFB01FF27E855FD4F8491E82FE71941
:103110005E9EC0011124B6010E947A2D80916A043E
:10312000689FB00111247A83B5CF0E94392EB50172
:103130000E948E2D8E159F050CF0ACCF83E0681693
:1031400088F00E94392EB5010E948E2D88830E943E
:10315000392E209169042695622F70E00E948E2DF1
:10316000280F2983909EF001919EF00D1124E45FB9
:10317000FD4F128280916A04893C58F088EC909E41
:10318000F001919EF00D1124E45FFD4F8483838351
:1031900081CF8431A0F784E1F2CF60916704669516
:1031A00070E04BE050E088E091E00E94492E892BCE
:1031B00019F481E0809365040E94A40B9093E103CD
:1031C0008093E00380916604846080936604089590
:1031D0009091670490FF3EC08115E9F18932E8F5CE
:1031E0008F77282F220F809167048170282B2093DE
:1031F000670480916604816080936604611581F0A4
:10320000309168044091690450916A0460916B04A4
:1032100070916C0480916D0490916E040E944D1425
:1032200060916704669570E04BE050E088E091E0C3
:103230000E94492E892B99F00E94220881E08093F8
:10324000E30320E040916A0460916904809168047E
:103250000E94C414089581E0C4CF88E2C2CF0E94C6
:10326000CD18ECCF8091670486958F5F893208F086
:1032700081E061E00E94E8180895809167048695D6
:103280008A9509F488E261E00E94E8180895909117
:10329000670490FF08C09695981728F0961718F4C1
:1032A0000E943219089561E00E94E8180895A0E094
:1032B000B0E0EDE5F9E10C942A2D8C01FC0184814C
:1032C0008115B9F161E0C8010E94C406EC01F80162
:1032D0008581C034FEE7DF0789F0811509F4A1C0BC
:1032E000809170048272FE01E053FC47E830F105E2
:1032F00008F097C0EA5BF04D0C94A22D8115F1F017
:103300000E94AE08909357048093560483EE0E9467
:10331000B30F809177048770811559F0F80185818A
:10332000811539F08091BE0482FF03C082E00E94C3
:103330004504CDB7DEB7E1E10C94462D83EE0E9443
:10334000071080915604909157040E94E1098E3B2A
:103350009105F8F680EE0E94B30FE0EAEE2EE6E06B
:10336000FE2EF7018491811509F44EC0813009F0D9
:1033700047C0E7012196FE018491813041F42196F6
:10338000FE0184910E94731021967E01EACF823063
:1033900039F4E7012296FE0184910E94B30FF4CF25
:1033A000833039F4E7012296FE0184910E940710D0
:1033B000EBCF843049F7E7012296FE01849120E0AB
:1033C00030E04AE0FE0131968053990B8A30910536
:1033D00060F021153105C1F28FE99FE00197F1F707
:1033E00000C0000021503109F4CF429FB001439F3B
:1033F000700D11249C01260F371F8491EF01E2CF3D
:103400000E940111E701C0CF80EE0E94071081CF1A
:10341000811521F08FEF03C08115E1F381E00E9457
:10342000200FF8015580511409F4CDC0D7FFCBC04F
:103430000E94AF0B8093590490915A04913029F463
:1034400081FF03C089E30E94731080917004809310
:103450005804109270041092760480915A048230BD
:1034600009F46EC0B8F4811164C082EE0E94B30FFB
:1034700017C010925A040E94190FD3CF81E0809395
:103480005A04F9CF82E0FBCF83E0F9CF84E0F7CF95
:1034900085E0F5CF843009F467C0853009F469C050
:1034A0004E01E89497F8A12CB12CEFE3FCE9319799
:1034B000F1F700C0000040905A045CE1C52ED12C09
:1034C00067E0E62EF12C7AE0672E712CD501C4015D
:1034D0000C2C04C0B695A795979587950A94D2F7BA
:1034E000F82FFF703F2E511479F024E04212A8C546
:1034F0003AE0F31708F4A4C580915A04823009F029
:1035000049C082E60E94731080915A04823009F00B
:1035100045C09AE08AEF830D391638F489E0830DAF
:1035200090E0B3010E948E2D875A0E947310512C97
:103530008EC560E070E088E193E00E943A10B0CF61
:103540008091590480FD03C083E50E94731082EED0
:103550000E94B30F8FE39CE90197F1F700C00000D0
:1035600087E50E9473109CCF86EE0E94731088E15D
:10357000F8CF60E070E08BE191E00E943A1060E0EB
:1035800070E085E290E00E943A1060E070E088E22E
:1035900090E0D3CF80E30E940111B6CF86EF830D78
:1035A000863028F080E3830D0E940111C0CF87E5AB
:1035B000FACF843009F456C0853009F455C08091A3
:1035C000580480937004F8018581811509F4CAC0FC
:1035D000C137FCE7DF0709F4B5C0C2372CE7D207D3
:1035E00009F4BAC0C0373CE7D30709F048C580905A
:1035F0005F019090600180915D0190915E0188165D
:103600009906C9F5809161048032A9F58BE594E0B3
:10361000EC01019628812032D9F38881811509F4C3
:1036200078CE813009F08BC099818A81913009F080
:1036300052C022960E9473102196EFCF8CE20E9416
:1036400073108091590481FFBACF89E30E947310EF
:10365000B6CF82EE0E9407108091590480FDAFCF53
:1036600083E5F4CF88E2F2CF60E070E088E290E09A
:103670000E943A10A4CF90925E0180925D0180E298
:1036800080936104A12CB12C1092600430E6E32EEB
:1036900034E0F32EC0E0D0E04AE0442E512C612CFF
:1036A000712CC501B401A30192010E94F62E605D48
:1036B000603339F4209729F089288A288B2809F467
:1036C00060E2F70162937F0149015A012196C530FA
:1036D000D10539F79BCF923021F422960E94B30F87
:1036E000ABCF933021F422960E940710A5CF9430DF
:1036F00011F02196A1CF229620E030E06AE0AE01E1
:103700004F5F5F4F8053990B8A30910568F0211508
:10371000310509F491CF8FE99FE00197F1F700C0DF
:10372000000021503109F3CF629FF001639FF00D3B
:1037300011249C012E0F3F1F8981EA01E0CF0E94D6
:1037400001117ACF80915F0190916001059690936D
:10375000600180935F01DDCD80915F0190916001F8
:103760000597F5CFFE01E851FC47E730F10508F079
:10377000DDC0E25BF04D0C94A22D26E241EE61EE3D
:103780000E949310C6CD27E245EE65EEF9CF26E202
:1037900041EE60EEF5CF27E245EE64EEF1CF26E292
:1037A00041EE62EEEDCF27E245EE66EEE9CF28E28C
:1037B00041E0EBCF8091BD0481608093BD046091B6
:1037C000BD047091BE0484E090E00E94AE2E0E9481
:1037D0005E119FCD8091BE0488608093BE04EFCFC0
:1037E0008091BD048260E9CF8091BD048460E5CF03
:1037F0008091BD048860E1CF8091BE048160EDCFEF
:103800008091BE048260E9CF8091BD048061D5CFF4
:103810008091BD048062D1CF8091BD048064CDCF02
:103820000E945E118091BD048068C7CF8091BD0465
:103830008C60C3CF8091BE048360CFCF8091BD04E4
:103840008E7FBBCF8091BE04877FC7CF8091BD04A0
:103850008D7FB3CF8091BD048B7FAFCF8091BD04AE
:10386000877FABCF8091BE048E7FB7CF8091BE049F
:103870008D7FB3CF8091BD048F7E9FCF8091BD049B
:103880008F7D9BCF8091BD048F7B97CF0E945E116F
:103890008091BD048F7791CF8091BD04837F8DCFC0
:1038A0008091BE048C7F99CF8091BD0482FB9927C3
:1038B00090F921E0922790FB82F990FB83F97DCF6C
:1038C0008091BE04982F909590FB80F990FB81F930
:1038D00084CF9091BD04892F8F7B96FF80646DCF3C
:1038E0000E945E119091BD04892F97FB87F9805843
:1038F00064CF61E08EE090E00E94902E60CF60E0A7
:10390000F9CF9091BD04892F8F7E94FF806155CFB0
:103910009091BD04892F8E7F90FF81604ECF909152
:10392000BE04892F877F93FF886057CFC6319CE7FD
:10393000D90709F590917004811599F0892F8A7A39
:1039400091E0811101C090E09093630465E38111DF
:1039500001C069E28EED91E00E9494080E943F0F41
:10396000D8CC80916304811521F085E30E9438044E
:10397000F5CF89E2FBCF811189C0809170048272FA
:10398000FE01E052F847E531F10508F094C0EB5A2A
:10399000F04D0C94A22D8091670480FF1EC0282F4B
:1039A0002E7F209367043091680440916904509100
:1039B0006A0460916B0470916C0480916D04909125
:1039C0006E040E944D140E9422088091660481605A
:1039D000809366040E94C00B9CCC81608093670436
:1039E00061E086950E94E81894CC4DE359E162E3CA
:1039F00079E10E9429088DCC42E359E16DE379E138
:103A0000F8CF49E655E16FE575E1F3CF4FE555E1B4
:103A100069E675E1EECF40E855E163E775E1E9CF8E
:103A200043E755E160E875E1E4CF4AE955E16DE827
:103A300075E1DFCF4DE855E16AE975E1DACF4AEA91
:103A400054E160E974E1D5CF40E954E16AEA74E1F8
:103A5000D0CF61E081E0C6CF65E082E00E944719E7
:103A600058CC68E086E0FACF6EE089E0F7CF64E1F9
:103A70008FE0F4CF67E185E1F1CF61E088E1B2CF7B
:103A800062E289E1EBCF68E283E2E8CFCA35ECE796
:103A9000DE0709F485C008F05CC0C1302CE7D2070E
:103AA00009F47CC0C3303CE7D30709F471C0C115E9
:103AB000DC4709F460C0F8018581E080F180811560
:103AC00009F472C0C7010E949006C82F682FC70171
:103AD0000E94C503B7018C2F0E9474040E947905CF
:103AE000D82FC92FF801B580A680A2942FE0A2227A
:103AF0008091770487708115F1F0EB2CB114E1F01F
:103B0000892F807F803451F080E28D0F883098F0CB
:103B1000A11004C0892F807E803269F08091BE049C
:103B200082FF09C082E00E9445048091770487707B
:103B3000EE24E3948111E12C8C2F82958F70C82E96
:103B4000D12C8C3008F095C0F601E659F04D0C945C
:103B5000A22DCB359CE7D90729F1CC35DC4709F0FC
:103B6000AACF8091BE0482FB882780F991E0892743
:103B70000E94020FA0CF0E945E11FFEF24E33CE001
:103B8000F15020403040E1F700C000000E94450E97
:103B90006FEF7FEF80E090E00E94AE2E0E948511D3
:103BA00081E0E6CF80E0E4CFC7010E94FB03C82F8D
:103BB00091CFFC2FFF70FF2EC03118F0F29490EFE0
:103BC000F922B114B9F0F11469F080E28D0F883058
:103BD00010F0D11109C0809170048F298093700476
:103BE0000E943F0F8D2F43C0809176048F298093D0
:103BF0007604F6CF8D2F0E940710F114D1F180E2E8
:103C00008D0F883010F0D11104C08F2D0E946104F7
:103C100006C0F094809176048F21809376040E94F0
:103C20003F0F27C02C2F2F70F22EC07FC03219F00B
:103C3000F29480EFF822D11551F0D13009F491C0FF
:103C4000B11409F49BC0A11409F442C0CBCF8091F8
:103C5000BE0482FD39C0B11489F1F11439F08091AC
:103C600070048F29809370040E943F0F80E00E94AF
:103C7000B30F28E0C21AD10834E0C316D10410F4FF
:103C80000E94AF0BE114A9F08091770480FD11C070
:103C9000F80115828695869586950E94A303C80132
:103CA0000E945719809177048695869586950E9483
:103CB000B30360E0C8010E94C4063BCB80E00E94D1
:103CC0000710F114B1F2A1CFB11469F1A11004C031
:103CD0008F2D0E949F0FCDCF31E0A31210C0C09155
:103CE0006F048F2D8C23F81621F20E94AE0890935A
:103CF0007B0480937A04CF29C0936F04BACF83E00A
:103D0000A812B7CF8F2D0E949F0F8F2D0E94D2082F
:103D1000809171049F2D9823F91609F4AACF8F2959
:103D200080937104A6CFA11012C08F2D0E948D0F19
:103D30008F2D0E94D208809171049F2D9823911598
:103D400009F497CFF094F822F092710492CF91E0A9
:103D5000A9128FCF809170048F21811509F489CF2A
:103D6000E4CFB11429F0E2E0AE1608F082CFB0CF74
:103D7000A1107FCF8F2D0E948D0F7BCFA114D1F387
:103D8000D93349F4FFEF27EE33E0F15020403040C3
:103D9000E1F700C000008D2F0E9407106ACF8C2F22
:103DA000869586958370811569F0813009F061CF21
:103DB0008D2F9C2F9370B11002C080E090E00E9484
:103DC0006E0857CF8D2F9C2F9370B11002C080E0EA
:103DD00090E00E9448084DCF6B2D8D2F0E94100956
:103DE00048CF8C2F8370811140C0B11042CF4D2F2E
:103DF000429546954770440F440F2D2F2F7030E0A9
:103E0000042E02C0220F331F0A94E2F780E090E0F4
:103E1000D4FF09C08FE090E002C0880F991F4A9537
:103E2000E2F780959095C695C695C370C230A1F013
:103E3000C33079F04091720450917304C13039F06D
:103E4000822B932B842395230E94990312CF242B3A
:103E5000352B822B932BF8CF822B932B209172043E
:103E60003091730482279327EFCFB11491F1C0FFF3
:103E700000CF4D2F429546954770440F440F2D2F8C
:103E80002F7030E0042E02C0220F331F0A94E2F795
:103E900080E090E0D4FF09C08FE090E002C0880F7E
:103EA000991F4A95E2F780959095C695C695C3707F
:103EB000C230C1F0C33099F0409174045091750440
:103EC000C13059F0822B932B842395230E949E03AB
:103ED000D0CE823008F4CDCECCCF242B352B822B04
:103EE000932BF4CF822B932B209174043091750483
:103EF00082279327EBCFCF70B11429F08C2F0E942B
:103F0000A3038D2FE6CE8D2F0E948D0F8C2F0E9444
:103F1000B303AFCED23F09F43EC060F4D03FB9F056
:103F2000D13F81F0B11409F47BC0A1105BCE8C2F7E
:103F30008F7135C0D33FB1F1D43FA1F78091BE045A
:103F400082FD3EC08C2F8F71B11409F328C0B114CB
:103F500099F0A1108ECECF7181E090E0FC0102C0FB
:103F6000EE0FFF1FCA95E2F7EF0180917404909164
:103F700075048C279D27AACFF2E0AF1608F079CE02
:103F8000CF7181E090E09C0102C0220F331FCA95DF
:103F9000E2F7E901EACF8C2F8F71B110B8CF0E9400
:103FA000A30367CE80E090E0B11409F48FCFCF7106
:103FB00081E090E002C0880F991FCA95E2F786CF92
:103FC000B114E9F0809177048770843061F4109225
:103FD000770410927904109278048C2F8F710E94CC
:103FE000B303E12C46CE33E0A316D8F7CF718C2F64
:103FF0000E94A30363E08C2F0E94BA08F2CF83E0F3
:10400000A81650F010927704109279041092780458
:1040100064E08C2F8F71F0CF81E00E944504E1CFE6
:10402000A11459F0D93309F0B6CE9FEFE7EEF3E0D3
:104030009150E040F040E1F7ACCE8C2F8F7167CF0C
:10404000311062CA84E0E816F1040CF45DCAE1E0C4
:10405000EE1AF108F4E0CF1AD1082FEFE216F206BB
:1040600009F034CA80915A04823009F4F2CA08F087
:10407000A0CA8111E3CA82EE0E940710A0CAFE0105
:10408000E851FC47E730F10508F473CB1092620465
:104090009E0130572332310508F048CC84E090E08F
:1040A0000E947A2E9093BE048093BD04FE01E150DD
:1040B000F047E232F10508F07DCBEA58F04D0C9460
:1040C000A22D8091BC04803178F48091BB048115CD
:1040D00059F0E0917D0420917C043091B704409127
:1040E000B60457E02E1301C008956E2F70E05E9F56
:1040F000F0011124DF01A258BB4F14968C91149744
:10410000811581F111968C91119783132BC08C919D
:10411000841328C015968C911597811123C012968F
:104120008D919C91A091B804B091B9048A1B9B0B0E
:10413000A0915F01B09160018A179B0798F480916C
:10414000BC048F7080618093BC04EC57FB4F80816E
:104150008F708061808386EB94E00E9457190E94E3
:104160002E040895FB013196E770BCCFADE0B0E0BE
:10417000ECEBF0E20C942E2D8C0186E0F801DE01D0
:10418000189601900D928A95E1F7F801E080F5808C
:10419000A280B380C48086EB882E84E0982E709035
:1041A000BA04711020C0C114D9F0F11409F421C16E
:1041B000C8010E94F306811509F41BC187E0F801CC
:1041C000D40101900D928A95E1F7F1E0CF1206C07B
:1041D0008091B6049091B7040E94E4060E94612089
:1041E000FF24F39456C0D090BB048091B804909102
:1041F000B9049501281B390BC90120915F01309149
:104200006001D11409F4BAC08217930708F090C076
:10421000C11431F39091B704C1808091BC04803106
:1042200008F058C0C91214C09091B6049E1110C075
:10423000F1104AC08F7080618093BC0486EB94E0DB
:104240000E9457198091BC04F8018683F12C21C08B
:10425000F1103AC040E06C2D8E2D0E94450B40E0DD
:104260006C2D8E2D0E94450BF82E8111EFCF888585
:1042700099850E94E406292F22952F70903470F4BE
:104280009F702230A0F09115B1F0F8019681903125
:1042900090F48F2D2D96EDE00C944A2D2A5F2F700F
:1042A000223068F0C8010E945719FD2CF2CF9115F9
:1042B00011F0811571F3805E883058F3F3CF803FA1
:1042C00040F3815F8330F9CF8091BC04816080939B
:1042D000BC04BCCFC91207C09091B6049E1103C0A4
:1042E000F11409F46FC0C8010E94F306811509F4A6
:1042F00080C0F11409F47DC08091BC04803278F054
:104300002091B6043091B7043A832983BC82AB82F2
:104310007D821E828F83CE0101960E94571987E00D
:10432000F801A6EBB4E001900D928A95E1F756CF23
:104330008091BC04803150F486EB94E00E945719C0
:1043400087E0F40111928A95E9F780CFC11409F44E
:1043500047CF2091B70491812913C5CF9091B6041E
:104360009E11C1CFF110BFCF8683C8010E9457199B
:1043700087E0F40111928A95E9F732CF821793070B
:10438000F8F6C11409F42CCFF11499F13091B70467
:104390002181321324C02091B6042E1120C08E3BFF
:1043A0009105A0F48091BC0480FD10C0803170F0B4
:1043B0008683982F907F903F31F0982F907F905F69
:1043C0008F70892B8683C8010E94571987E0F801F6
:1043D000A6EBB4E001900D928A95E1F701CFC801F8
:1043E0000E94F30681119BCF8091BC048160809371
:1043F000BC04C8010E945719F3CEABE1B0E0E3E082
:10440000F2E20C94382D4E8B5F8B688F798F8A8FF8
:104410009B8F9111109276041D8A86E0FE0176969C
:10442000DE011F9601900D928A95E1F78091BE04FE
:1044300082FF1FC00E94AE08209178043091790459
:10444000821B930B8838934138F08091770482FD6A
:1044500003C082E00E9445040E94AE0820917A04C5
:1044600030917B04821B930B8838934110F00E949B
:1044700069048B89811529F061E0CE010F960E94B5
:10448000C40687E0FE013F96DE01189601900D926A
:104490008A95E1F7CE0108960E94B620811110C0DE
:1044A00087E0FE013896DE01119601900D928A9503
:1044B000E1F720917C0440917D048C8581110BC033
:1044C00017E080917D0490917C0489132DC06B9638
:1044D000E3E00C94542D30E0C901019687709927D0
:1044E0004817190671F40E945E1110927C04109214
:1044F0007D0487E0E6EBF4E0DF011D928A95E9F7A1
:10450000DFCF97E0929FD001939FB00D1124A25866
:10451000BB4FFE01319601900D929A95E1F7809381
:104520007C040E942E04CCCF189FC0011124825815
:104530009B4F0E94B620811551F280917D0490E03E
:1045400001968770992780937D04BBCFA6E0B0E0E9
:10455000ECEAF2E20C94372D0E94AE088C018091B7
:10456000290490912A048017910779F019821A8200
:104570000E94AE08BC0149815A8180E090E00E940F
:10458000FD2110932A04009329042696E4E00C945C
:10459000532DA3E1B0E0EFECF2E20C942E2DFE01DE
:1045A0003C9688E0DF011D928A95E9F78EE1A82EFE
:1045B00081E0B82E8F014F01EE24E394F12C2EE11F
:1045C000C22E21E0D22EF50181915F018F3F09F4C7
:1045D00041C0F894E82FE295EF70F0E021A18F70D0
:1045E000A70102C0440F551F8A95E2F7CA01922F16
:1045F000982B91A392A18095892382A3789400C0DF
:10460000E8E1F1E031E0712C21912F3F89F0A22FF8
:10461000A295AF70A05EB0E08C9190E02F7002C0C8
:10462000959587952A95E2F78170811509F49AC0CE
:1046300080E0782A330FCE16DF0631F7F501319787
:1046400080818F3F11F00E941D0750EA5A95F1F7C3
:10465000D8017C920F5F1F4FB2E2AB16B1E0BB06F0
:1046600009F0B1CF48E050E0B4018EEB93E00E9436
:10467000562E892B09F078C00091C7038091EF0175
:104680008115F1F08091ED019091EE010E94E10918
:104690000597B0F010E004531C4F44E050E06EEB7F
:1046A00073E0C8010E94562E892B41F084E0EEEBA6
:1046B000F3E0D80101900D928A95E1F71092EF0195
:1046C0000E94640BE091C7039E012F5F3F4F790169
:1046D000811509F492C084E0D9011D928A95E9F709
:1046E0000E2F10E004531C4F8091F0018A3008F027
:1046F0004FC046EA56E1B701C8010E94C80E8115B5
:1047000009F469C04AED56E1B701C8010E94C80E1C
:10471000811509F460C043E357E1B701C8010E9465
:10472000C80E811509F457C04AE857E1B701C8011E
:104730000E94C80E811509F44EC01092F0018091BC
:10474000C60390E044E050E0B70184539C4F0E94C0
:10475000562E21E02093EC01892B79F56396EDE04C
:104760000C944A2D832F65CF88E0F401AEEBB3E0C3
:1047700001900D928A95E1F70091C70381E0809343
:10478000EF010E94AE089093EE018093ED017ACF85
:104790008091EA019091EB010E94E109843F9140F0
:1047A00008F0A7CF8091EC018115C1F284E0F701F8
:1047B00011928A95E9F71092EC01E091C603F0E0BE
:1047C000E453FC4F89819A81AB81BC8180839183C2
:1047D000A283B383C3CF8091F0018F3F39F40E944D
:1047E000AE089093EB018093EA01DCCF8F5F80935A
:1047F000F0018A3008F4A3CFF2CFF0E0E453FC4F8D
:1048000080819181A281B38180930E0490930F04E3
:10481000A0931004B093110464E070E08EE094E083
:104820000E94300880930D044091E90350E06091AC
:10483000E80370E066507C4FC7010E94632E8981B7
:104840008093130461E070E0C7010E9430088093F8
:1048500012048090140490901504A0901604B09057
:1048600017048091E6019091E701A091E801B091D1
:10487000E90188169906AA06BB06D1F08092E601E6
:104880009092E701A092E801B092E9010E94640BC6
:1048900081110EC00E94D509861A970AA80AB90A82
:1048A0008092250490922604A0922704B0922804B6
:1048B0008BE0E8E1F4E0D70101900D928A95E1F7F1
:1048C000809118048695F0901904E0901A04D09015
:1048D0001B0400912104109122041092220411154E
:1048E00009F43CCF10FF0BC029819091670420FF91
:1048F0001AC091609093670460E00E94E81811FF6D
:1049000006C020E04D2D6E2D8F2D0E94C41412FF85
:1049100004C00115A9F00E94CD1813FF1FCF81E03C
:104920008093E3031BCF9E7F909367040E9422082D
:10493000809166048160809366040E94C00BDFCF83
:104940000E942208EACFCDB7DEB728970FB6F894B9
:10495000DEBF0FBECDBF85B7806885BF85B78068D5
:1049600085BF84B7877F84BF0FB6F894A8958091E0
:104970006000886180936000109260000FBE80E844
:1049800090E00FB6F89480936100909361000FBEA1
:104990008BE197E09093DD018093DC010E949B0AFC
:1049A0000E94EA0A8091E20084608093E200789499
:1049B00080912304811599F08091E9001091EC0019
:1049C0001795112717958F70182B1092E900809179
:1049D000E80083FD0E949B111F701093E90082E0A4
:1049E00084BD93E095BD9AEF97BD80936E001092C1
:1049F000250410922604109227041092280484980B
:104A00008C988FE891E00197F1F700C000008FB11A
:104A1000829581708093220180912201811107C1CA
:104A20008BE1809313018BE1809314010E94640B4E
:104A300081110E94C62B9091220181E0292F282705
:104A40002093E8039093FC03909122018093E90363
:104A5000909122018093F90380912201811106C077
:104A600086EF80932C0187EF80932B0180912C019E
:104A7000E82FE295EF70A1E2AE0FB0E04C918F709D
:104A800021E030E0B90102C0660F771F8A95E2F796
:104A9000CB01962F909594239C93EE5DF0E090814E
:104AA000892B808380912B01E82FE295EF70A1E2A2
:104AB000AE0FB0E04C918F70B90102C0660F771F46
:104AC0008A95E2F7CB01962F909594239C93EE5D07
:104AD000F0E09081892B80838FE891E00197F1F7D6
:104AE00000C000001091E9036CE271E04BE251E07C
:104AF0002AEEE22E23E0F22EFB018E2F861B811779
:104B000008F497C08091220181111EC081E3809337
:104B10001E0183E380931F0182E38093200186E3DB
:104B20008093210186E0E1E6F1E0DE01119601903B
:104B30000D928A95E1F786E0FE013196A8E1B1E099
:104B400001900D928A95E1F78091220191E08927E9
:104B5000880F880F8093C70394E0981B9093C60337
:104B60000EE111E092E2E92E91E0F92EF801819137
:104B70008F018F3F11F00E941D07E016F106B1F77B
:104B800008E111E08EE1E82E81E0F82ED8018D9148
:104B90008D018F3F11F00E941D07E016F106B1F75D
:104BA00088E0ECECF3E0DF01282F1D922A95E9F76D
:104BB000EEEBF3E0DF011D928A95E9F780E090E0EB
:104BC0000E947A2E863E9E4F11F00E94A71582E029
:104BD00090E00E946C2E8093D40384E090E00E94C9
:104BE0007A2E9093BE048093BD040E94C922EFEFF9
:104BF000F6E721E0E150F0402040E1F700C000007E
:104C00000E94C922EFB1E295E17081E0E827EE0F42
:104C1000EE0FF0E0E453FC4F808185FF32C06FEF70
:104C20007FEF80E090E00E94AE2E0E94450E80E073
:104C3000F8CE0191802F82958F70805E90E0DC012C
:104C40002C91DA013D91AD01832F82958F70805EAA
:104C500090E0DC018C9190E03F7002C095958795C3
:104C60003A95E2F78170880F30E00F7002C03595F9
:104C700027950A95E2F72170822BD7018D937D014C
:104C80003CCF83E090E00E946C2E90E00E9499035C
:104C90008CE090E00E946C2E80935A04843009F4DA
:104CA00015C1811509F416C1813009F415C110929E
:104CB000C80384E080935A048091C903811192C093
:104CC00080E090E00E947A2E863E9E4F21F00E9466
:104CD000A7150E94731488E090E00E94742E6B0167
:104CE0007C0184E290E00E946C2E282F30E040E0AE
:104CF00050E060E070E080E090E000E20E94B72DBC
:104D0000E22FA32EB42EB52FA62FF72F97018601E1
:104D100040E050E0BA01EC29A12AB22AB32BA42B1F
:104D2000F52B862B972BE0936704A0926804B09232
:104D30006904B0936A04A0936B04F0936C048093AD
:104D40006D0490936E048091660483608093660482
:104D5000E230C8F50E94731488E090E00E94742E3F
:104D60006B017C0184E290E00E946C2E282F30E0E1
:104D700040E050E060E070E080E090E000E20E94FF
:104D8000B72D5901B42FA52FF62FE72F97018601D4
:104D900040E050E0BA01AC28B12AB22BA32BF42B8F
:104DA000E52B862B972BA0926704B0926804B093F2
:104DB0006904A0936A04F0936B04E0936C048093FD
:104DC0006D0490936E040E940D080E942208809149
:104DD000670480FF04C060E086950E94E81881E0C7
:104DE0008093C9030E94640B811102C00E94C92BE9
:104DF00083E291E090932C0480932B04FDEDCF2E61
:104E0000F3E0DF2EA4E06A2E712CCE010196B8E10A
:104E1000AB2EB12C8F83988780912304853049F481
:104E200080912304853009F459C00E945E110E94CC
:104E3000AF0B0E94C92205ED13E0ECECEE2EE3E08F
:104E4000FE2ED701F80191918D91CE16DF0609F45F
:104E500095C09817C1F30E94640B282E912CD7019E
:104E60008D907D01F80131908F01381441F1382483
:104E7000512C44244394842D83218115C1F02114A5
:104E8000B1F059829A820E94AE089C838B83F1E034
:104E9000FD8391E0842D8821811101C090E09E83E3
:104EA00049815A816B817C818D810E94FD215394BF
:104EB000440C26E05212DFCFF801319780829394A0
:104EC00048E09412CCCF0E94870B5CC080E08093B6
:104ED000C803F2CE81E0FBCF82E0F9CF80912304BA
:104EE000843011F11092CA0360E40FB6F894A895CB
:104EF000A09260000FBE6093600083B7817F8460E2
:104F000083BF83B7816083BF7894889583B78E7F92
:104F100083BF0FB6F894A895809160008861809354
:104F20006000109260000FBE8091CB03811509F4E0
:104F300077CF0E94C922ECECF3E084ED93E021915D
:104F4000211104C08E179F07D1F76ACF80E189BD78
:104F500082E189BD09B400FEFDCF8091D8008F7D2C
:104F60008093D8008091E00082608093E00080917F
:104F7000E00081FDFCCF0E945E1152CF98136BCFF1
:104F80000E94A6220E94640B80916504811509F499
:104F90006CC080916404E0916704E695E81BE0939F
:104FA000E2038F3009F49AC008F062C0863009F439
:104FB0007EC0893009F486C0823009F46DC000EDEE
:104FC00017E076E3E72E77E0F72E8091E303811573
:104FD00061F01092E3030E94A40B9093E10380938D
:104FE000E0031092E5031092E4030E94A40B9C01DD
:104FF0008091E0039091E103A901481B590B4F3FB9
:105000005F4798F54091DF034115B1F01092DF033F
:105010004091DD035091DE03241B350B2F3F3F47AA
:1050200058F4405D5A485093DE034093DD032091CD
:1050300066042860209366048090E4039090E50362
:10504000800F911F9093E1038093E00380EE93E043
:10505000F70109958091E4039091E503892B29F4E8
:10506000892819F081E08093DF03E12C912CCFC0D7
:10507000883109F44FC0833209F43CC0853109F00E
:105080009ECFF0E0E055FB4FE4910E2F10E026EDAF
:10509000E22E2CE0F22E99CFF0E0E454FB4FE491A5
:1050A0000E2F10E061E2E62E6EE0F62E8ECFF0E0DD
:1050B000E754FB4FE4910E2F10E055E3E52E5EE040
:1050C000F52E83CFE695F0E0EA54FB4FE4910E2FE6
:1050D00010E042E1E42E4CE0F42E77CFE695F0E0CC
:1050E000ED54FB4FE4910E2F10E030E5E32E3CE051
:1050F000F32E6BCF8E2F63E00E94602DE92FF0E03E
:10510000E355FB4FE4910E2F10E09DEFE92E97E160
:10511000F92E5BCF08E210E089E5E82E8DE0F82E4D
:1051200054CF0E2D10E0F801E45DFE4F4081E42FD6
:10513000E295EF70E05EF0E02081F801E55DFE4F62
:105140003081E32FE295EF70E05EF0E0808190E047
:105150003F7002C0959587953A95E2F78170880F68
:1051600030E04F7002C0359527954A95E2F72170DF
:10517000822BD801A651BC4FEC919E2F93708917BA
:1051800009F444C0EE0FEE0FE82BEC93F090E80327
:10519000FE0CEF70F0E0EC56FE4F0A511C4F808180
:1051A000D8019C91890F8C9320E0843084F0EF2DFE
:1051B000F0E0E650FC4F80818F5F80830E94640B9B
:1051C000811521F060E08F2D0E94F11021E0F8019F
:1051D00080818D3F84F4EF2DF0E0E650FC4F80811C
:1051E000815080830E94640B811521F061E08F2D36
:1051F0000E94F11021E0D8018C91082E000C990B2F
:10520000B3010E948E2DF8018083922AE39480914D
:10521000E903E81608F485CF91100E94A10B86E0FF
:10522000E0E5F4E0AF81B88501900D928A95E1F751
:105230001092520410925304109254041092550488
:105240008B819C81892B811509F44BC08091EE03E1
:105250009091EF030E94E1099C0180914E04811519
:1052600009F4C9C025313105E0F18F3F19F08F5F96
:1052700080934E041B81111559F00E94370791E06D
:1052800011160CF09FEF899F802D112480935204FA
:105290001C81111559F00E94370791E011160CF08E
:1052A0009FEF899F802D11248093530430915204E5
:1052B0003115B9F020915304211599F045EB3403D1
:1052C000C0011124892F911101C081E08093520403
:1052D00065EB260390011124311509F47FC030934A
:1052E00053048D819E81892B811509F44AC08091D8
:1052F000EC039091ED030E94E1099C0180914D0423
:10530000811509F473C021353105D8F18F3F19F0AB
:105310008F5F80934D041D81111559F00E9457072E
:1053200091E011160CF09FEF899F802D112480933E
:1053300054041E81111559F00E94570791E011166F
:105340000CF09FEF899F802D11248093550430919C
:1053500054043115B1F020915504211591F075EBED
:105360003703C0011124892F911101C081E080937E
:10537000540445EB240390011124311599F1309325
:10538000550446E050E06F81788580E594E00E9406
:10539000562E892B61F48091520490915304892BED
:1053A00090915404892B90915504892B81110E946E
:1053B000E80886E0EF81F885A0E5B4E001900D9261
:1053C0008A95E1F70E94AF0B9091F003891709F4D9
:1053D00023CD8093F0030E94D5091ECD81E08093F8
:1053E00053047FCF81E080935504CBCF2B30310520
:1053F00008F08ECFC6CF2B30310508F038CF71CFF3
:105400001F921FB61F9211248F939F93AF93BF9348
:105410008091CA03811113C08091090490910A04FC
:10542000A0910B04B0910C044196A11DB11D809375
:10543000090490930A04A0930B04B0930C04BF9149
:10544000AF919F918F911F901FBE1F9018957894D8
:105450001F921FB61F9211248F939F93AF93BF93F8
:105460008091090490910A04A0910B04B0910C045E
:105470000196A11DB11D8093090490930A04A09385
:105480000B04B0930C04BF91AF919F918F911F902B
:105490001FBE1F9018951F920F920FB60F921124E6
:1054A0002F933F934F935F936F937F938F939F932C
:1054B000AF93BF93EF93FF938091E10082FF09C008
:1054C0008091E20082FF05C08091E1008B7F809394
:1054D000E1008091DA0080FF24C08091D80080FF35
:1054E00020C08091DA008E7F8093DA008091D9000D
:1054F00080FF9BC080E189BD82E189BD09B400FEC7
:10550000FDCF81E0809323048091F601811109C0D1
:105510000E949B0A0E94EA0A8091E20084608093C4
:10552000E2008091E10080FF17C08091E20080FFDF
:1055300013C08091E2008E7F8093E2008091E200B0
:1055400080618093E2008091D80080628093D800CF
:1055500019BC85E0809323048091E10084FF29C079
:105560008091E20084FF25C080E189BD82E189BD90
:1055700009B400FEFDCF8091D8008F7D8093D800C4
:105580008091E1008F7E8093E1008091E2008F7E28
:105590008093E2008091E20081608093E20080913C
:1055A000F501811509F447C084E0809323048091BC
:1055B00023048091E10083FF27C08091E20083FFF4
:1055C00023C08091E100877F8093E10082E0809397
:1055D00023041092F5018091E1008E7F8093E10019
:1055E0008091E2008E7F8093E2008091E2008061F2
:1055F0008093E20042E060E080E00E94BA0A80917D
:10560000F00088608093F000FF91EF91BF91AF911F
:105610009F918F917F916F915F914F913F912F91CA
:105620000F900FBE0F901F90189519BC1092230475
:105630001092F60176CF8091E30087FF02C083E0ED
:10564000B4CF81E0B2CF1F920F920FB60F92112408
:10565000FF920F931F932F933F934F935F936F93FB
:105660007F938F939F93AF93BF93CF93DF93EF93EA
:10567000FF9309EE10E0F8018081C091EC00C7951E
:10568000CC27C7958F70FC2EF82A1082C0EFD0E08F
:105690008881877F888378940E949B11F80110820B
:1056A000888188608883CF2DCF70C083FF91EF9170
:1056B000DF91CF91BF91AF919F918F917F916F912A
:1056C0005F914F913F912F911F910F91FF900F90FC
:1056D0000FBE0F901F9018958EE14A9B02C08A95CD
:1056E000E1F74A9BFECF08955A9880E28A95F1F738
:1056F0005A9A0895FC013BE03A95F1F798E020E0D2
:1057000080E031E040E14A95F1F7880F4A9B02C002
:105710008160232742E04A95F1F7000040E14A9575
:10572000F1F79A9579F790E19A95F1F799B132E00E
:105730003A95F1F7000040E14A95F1F792FB99277D
:1057400090F992272081920F90830895A1E0B0E014
:10575000ECEAFBE20C94352D19828C017C01E60EFB
:10576000F11C0E151F0541F481E09981911180E033
:105770002196E6E00C94512D0E946C2BCE010196EF
:105780000E947A2BF80181938F01EBCF529A5A9A9B
:10579000089552985A9AEA9AE9E6F0E080818F7C5F
:1057A000808308956150770B91E001C0990F6A954D
:1057B000EAF7692F90E021E0611108C0911599F096
:1057C0005A9A80E28A95F1F75A980895362F38232D
:1057D000311539F05A9A922730E23A95F1F76695E9
:1057E000EBCF5A98F9CF5A98ECCFFF920F931F93B3
:1057F000CF93DF93EC018C01060F111DC017D10769
:1058000029F4CDB7DEB7E5E00C94522DF9900E9453
:10581000742B68E08F2D0E94D22BF0CF1F920F9235
:105820000FB60F9211240F931F932F933F934F9313
:105830005F936F937F938F939F93AF93BF93EF93F8
:10584000FF93CF93DF930F92CDB7DEB719820E94FB
:105850006C2BCE0101960E947A2B082F0695069597
:105860000695982F92959570202F2570920F292FCD
:10587000237096959695920F982797708981892B1A
:10588000811509F05CC0073008F059C080E18A95A5
:10589000F1F75A9A529A82E08A95F1F700C05A9825
:1058A00088E0089F80011124D801A35DBE4F1696A1
:1058B000ED91FC9117973097A9F06091A401709138
:1058C000A50114962D913C911597260F371F11961F
:1058D0008D919C911297680F791F13964C91139795
:1058E0008C910995F801E35DFE4F6381611551F0DC
:1058F0002091A4013091A50184819581820F931F8D
:105900000E94F52B0E94742B80E18A95F1F75A983A
:1059100052985A9A80E18A95F1F7F801E35DFE4FBB
:105920006081611551F02091A4013091A501818120
:105930009281820F931F0E94A62B0E946C2B0F90C6
:10594000DF91CF91FF91EF91BF91AF919F918F9197
:105950007F916F915F914F913F912F911F910F9187
:105960000F900FBE0F901F9018950F931F93CF931A
:10597000DF938C0107970CF064C0F894529A5A9800
:1059800085E08A95F1F70000C02FC695C570802F7D
:105990008570C80F8C2F8370C695C69593E0000F55
:1059A000111F9A95E1F7C80FC8018C2BEC010E94DA
:1059B000742B00C068E08C2F0E94D22B90E19A9546
:1059C000F1F752985A9A4A9B35C087E090E04A997D
:1059D00033C0F801E35DFE4F6381611561F02091F2
:1059E000A4013091A50184819581820F931F0E94AB
:1059F000A62B811519F10E946C2B80E28A95F1F794
:105A00005A98529A90E19A95F1F7F801E35DFE4FAA
:105A10006081611551F02091A4013091A50181812F
:105A20009281820F931F0E94F52B0E94742B789411
:105A300081E008C000C0C7CF019749F4529A5A9A32
:105A4000789480E0DF91CF911F910F91089500C06D
:105A5000BECF2F923F924F925F926F927F928F9222
:105A60009F92AF92BF92CF92DF92EF92FF920F93ED
:105A70001F93CF93DF93CDB7DEB7CA1BDB0B0FB6F7
:105A8000F894DEBF0FBECDBF09942A8839884888B4
:105A90005F846E847D848C849B84AA84B984C8844A
:105AA000DF80EE80FD800C811B81AA81B981CE0F41
:105AB000D11D0FB6F894DEBF0FBECDBFED01089526
:105AC000991B79E004C0991F961708F0961B881F50
:105AD0007A95C9F78095089587FB082E062687FDDD
:105AE000819567FD61950E94602D0EF4919507FCEC
:105AF00081950895AA1BBB1B51E107C0AA1FBB1FBC
:105B0000A617B70710F0A61BB70B881F991F5A9549
:105B1000A9F780959095BC01CD01089597FB072EBC
:105B200016F4009407D077FD09D00E947A2D07FC67
:105B300005D03EF4909581959F4F0895709561959D
:105B40007F4F0895EE0FFF1F0590F491E02D09940B
:105B50000E94182F332312F48A1B9B0B0C94B22D36
:105B60000E94182FB7FF0895821B930B0895002EF3
:105B7000083090F0982F872F762F652F542F432FC2
:105B8000322F22270850F4CF220F331F441F551FF6
:105B9000661F771F881F991F0A95B2F7002D089579
:105BA00097FD1094002E083098F00850232F342FC2
:105BB000452F562F672F782F892F912DF4CF1594CD
:105BC0009795879577956795579547953795279535
:105BD0000A95AAF71124002D08958F929F92AF92F3
:105BE000BF92CF92DF92EF92FF92CF93DF93EC01BF
:105BF000688179818A819B81611571058105910593
:105C000021F464E279ED8BE597E02DE133EF41E09B
:105C100050E00E94C42E49015A019B01AC01A7EA41
:105C2000B1E40E94E32E6B017C01ACEEB4EFA50160
:105C300094010E94F12EDC01CB018C0D9D1DAE1D47
:105C4000BF1DB7FF03C00197A109B048888399839E
:105C5000AA83BB839F77DF91CF91FF90EF90DF9076
:105C6000CF90BF90AF909F908F9008950E94ED2DA0
:105C7000089580E091E00E94ED2D0895A0E0B0E04D
:105C80008093000190930101A0930201B09303015E
:105C90000895FC014150504030F001900616D1F7B4
:105CA0003197CF010895882799270895FB01DC01DA
:105CB00004C08D910190801921F441505040C8F7E3
:105CC000881B990B0895FB01DC0102C001900D9225
:105CD00041505040D8F70895F999FECF92BD81BD4B
:105CE000F89A992780B50895A6E1B0E044E050E025
:105CF0000C94B62EA8E1B0E042E050E00C94B62E31
:105D0000DC01A40FB51F4150504048F0CB01840F77
:105D1000951F2E910E94912E41505040D0F708952A
:105D2000262FF999FECF92BD81BDF89A019700B454
:105D3000021639F01FBA20BD0FB6F894FA9AF99AF4
:105D40000FBE08950396272F0E94912E0E94902E39
:105D5000252F0E94912E242F0C94912E0196272FEF
:105D60000E94912E0C94902EDC01CB01FC01F9993C
:105D7000FECF06C0F2BDE1BDF89A319600B40D9297
:105D800041505040B8F70895052E97FB1EF400943B
:105D90000E94DB2E57FD07D00E94F62E07FC03D091
:105DA0004EF40C94DB2E50954095309521953F4F45
:105DB0004F4F5F4F089590958095709561957F4FF7
:105DC0008F4F9F4F08950E94182FA59F900DB49F4D
:105DD000900DA49F800D911D11240895B7FF0C9480
:105DE000E32E0E94E32E821B930B0895A1E21A2E4C
:105DF000AA1BBB1BFD010DC0AA1FBB1FEE1FFF1F6F
:105E0000A217B307E407F50720F0A21BB30BE40BBE
:105E1000F50B661F771F881F991F1A9469F7609505
:105E20007095809590959B01AC01BD01CF010895BF
:105E3000A29FB001B39FC001A39F700D811D1124CB
:105E4000911DB29F700D811D1124911D0895F8942C
:105E5000FFCF1C09240927092D09420942094209DB
:105E60004209420942094209420930093509390902
:105E70003F09500956095A0978129F12A5129F121C
:105E8000A512F8121A13A51218142514081A0C1AC0
:105E9000391A3E1A421A441A461A481AC71BCB1B13
:105EA000BD1BC31BCF1BD31BD71BCB1CF51CFC1C62
:105EB000011D061D0B1D101D151D1A1D1F1D241D66
:105EC000291D2C1D311D341D371D3A1D3D1D401D42
:105ED0008919431DD91DD91D121E121ECF1EEC1E7D
:105EE000391E391EF11E7B1F8A1F8A1F1E1C881C2B
:105EF000261CF01BF41B2A1CF81B2E1C3A1C041C2D
:105F0000811C081C3E1C0C1C421C691C101C461CDD
:105F1000701C161C4C1C541CFC1B321C001C361C18
:105F20001A1C501C601C791C7F1CEA1B221C8F1C35
:105F3000010000000101010201191A1B1C1D1E1F96
:105F4000202122003600363632363331F7F697C636
:105F5000343501F009A30EBA0EC10E66940000009C
:105F6000010000000000000004010000000000002B
:105F70000105000000000000010600000004070009
:105F800000000000000B0B000000000000FF00BE3E
:105F900000946697C634350000010202020206062C
:105FA000060909090909090F0F0F0F0F0F1515151C
:105FB0001819191919191919191919232323232320
:105FC0002304000100FF0100010000FFFF000001A9
:105FD0000001FF000D04E200E900EA00B500B60090
:105FE000B700CD008301CC008A0192019401210207
:105FF000230224022502260227022A02B300B4004B
:0C6000006F0070009F01CB019F02A00206
:00000001FF
